:100000000EC015C014C014C012C011C010C00FC063
:100010000EC019C00CC00BC00AC009C008C0112412
:100020001FBECFE5D2E0DEBFCDBF23D027C0E8CFD3
:100030001F920F920FB60F921124C09A0F900FBE0D
:100040000F901F9018951F920F920FB60F921124C8
:10005000C0980F900FBE0F901F90189580B78168C1
:1000600080BF89B7806689BF82E38EBD8AE08BBD81
:100070000895B89AB9987894F1DFFFCFF894FFCF3C
:00000001FF
